:020000020000FC
:100000000FC0AEC0C7C006C107C1DBC006C106C174
:0E00100006C101C1D4C0D4C003C103C103C1E5
:10002000F89405E401BF00E810E006BD16BD05E246
:1000300008BB02E107BBB0E0A0E6D2E0C0E600E00A
:100040000D93BD17E9F7AC17D9F712E00FE51EBF06
:100050000DBF00E000BD00E00BBF00E009BF08E0FD
:1000600005BB00E60ABF06E408BF01E005BF00E0EB
:100070000ABD03E003BF00E002BF00E009BD00E0ED
:1000800008BD00E60CBD00E00EBD00E00BBD00E5C4
:100090000DBD00E007BD05E600BF03EB07B900E0BA
:1000A00003B907EE06B908E004BB00E808B9A89553
:1000B0000EE119E301BD11BD00E60BBF01E005BB78
:1000C00000E009BF00E0102EE02EF4E0E0E002E3E3
:1000D000202E1AE000E0109376000093750090E067
:1000E000789404E6A89590FF03C09E7F0A95D1F707
:1000F000A89590FFFDCF9E7FF4E0E0E010E0009136
:10010000620030E020916500020F131F31E02EE005
:10011000021B130B17FD00E091FD069592FF00E016
:100120000BBD10E00091620030E020916500021BE1
:10013000130B30E02EE1020F131F17FD00E091FDBD
:10014000069592FF00E00EBD04B105B10F3908F429
:10015000926000916200083710F49D7F9460C8CFD0
:10016000FFB60F931F930AE0502E4E2C3E2CB299EF
:1001700004C002B70093600009C002B70093610099
:1001800010916000011B0093620091601F910F911C
:10019000FFBE1895FFB60F931F93B09904C002B726
:1001A0000093630008C002B70093640010916300DD
:1001B000011B009365001F910F91FFBE18951895C4
:1001C0001895FFB6F03019F4E03009F402C0319709
:1001D0001FC0709176006091750008946E097E09C9
:1001E000709376006093750039F47AE060E0709364
:1001F00076006093750000C0713030F462E0609367
:100200002900E092280004C0E0922900E092280032
:10021000FFBE189518951895189518951895189566
:10022000189518951895101718F4021708F400007F
:100230000895201B310B20F4041B150B08F400005B
:1002400008954F935F936F93551B441B61E110F426
:10025000400F511F57954795379527956A95B9F7E0
:100260005F934F933F932F930F911F912F913F9146
:100270006F915F914F9108954F935F936F934427D0
:10028000552760E1000F111F441F551F42175307E8
:1002900018F00395421B530B6A95A1F75F934F9398
:1002A0002F913F916F915F914F9108951F93E19925
:1002B000FECF10E01CBB10E01FBB8EBB0DBB753A20
:1002C00011F4E29AE19A1F9108951F93E199FECFEC
:1002D00010E01FBB8EBBE09A0DB31F9108951F93D2
:1002E0002F932BE11FE41A95F1F72A95D9F70A9578
:0802F000C1F72F911F91089541
:00000001FF
